:100000000C9484000C94A3000C94A3000C94A30003
:100010000C94A3000C94A3000C949A010C94A300DC
:100020000C94A3000C94A3000C94A3000C94A300C4
:100030000C94A3000C94A3000C94A3000C94A300B4
:100040000C94A3000C94A3000C94A3000C94A300A4
:100050000C9461090C94A3000C94A3000C94A300CD
:100060000C94A3000C94ED100C94B4060C94A30013
:100070000C94A3000C94A3000C94A3000C94A30074
:100080000C94A3000C94A3000C94A3000C94A30064
:100090000C9444120C9470060C94A3000C94A300CE
:1000A0000C94A3000C94A3000C9421010C94A300C5
:1000B0000C94A3000C94A3000C94A3000C94A30034
:1000C0000C94A3000C94A3000C94A300494E464941
:1000D0004E4954594E414ECDCCCC3D0AD7233C1706
:1000E000B7D13877CC2B329595E6241FB14F0A0053
:1000F0000020410000C84200401C4620BCBE4CCA43
:100100001B0E5AAEC59D740011241FBECFEFD1E265
:10011000DEBFCDBF1DE0A0E0B2E0E0EAFCE400E01D
:100120000BBF02C007900D92AE31B107D9F710E1B5
:10013000AEE1BDE001C01D92A83BB107E1F70E940E
:10014000801C0C944E260C9400008A3010F480938E
:10015000460E08951092420E1092430E1092440ED5
:100160001092450E08951092420E1092430E109276
:10017000440E1092450E1092460E82E08093470E78
:100180004FEF4093840E30E13093850E21E02093B1
:10019000860E88E998E09093880E8093870E1092DF
:1001A000890E40938A0E30938B0E20938C0E909381
:1001B0008E0E80938D0E30938F0E2093480E1092EA
:1001C000490E1092930E80E090E0FC01EE0FFF1FAD
:1001D000E65BF14F11821082019688309105A9F7F4
:1001E00080E090E0FC01EE5BF14F808F019688305B
:1001F0009105C1F780E090E024E6FC01EE5BF14F51
:1002000020A3019688309105C1F78FEF9FE390936B
:100210007B0E80937A0E90937D0E80937C0E88E007
:1002200080937E0E8FEF9FE19093800E80937F0EE0
:100230008CE291E09093820E8093810E1092830E57
:1002400008951F920F920FB60F920BB60F921124C2
:100250002F933F934F935F936F937F938F939F93CE
:10026000AF93BF93EF93FF931092A5001092A40059
:100270002091220230912302E091470E8091950D4A
:10028000F0E044E0EE0FFF1F4A95E1F7E80FF11DA3
:10029000EC5DFD4F8081280F311D3093A900209324
:1002A000A8008091220D863034F08FEF90E090937B
:1002B000A9008093A800A8950E9493100E94FB03B8
:1002C000E091460E8091950DF0E034E0EE0FFF1FB7
:1002D0003A95E1F7E80FF11DEC53FD4F81E06081A5
:1002E0000E94120480E293E00197F1F78091220DC1
:1002F0008F5F8093220D86E00E948C048F71809323
:10030000230D6091220D4091950D0E949510FF9153
:10031000EF91BF91AF919F918F917F916F915F917D
:100320004F913F912F910F900BBE0F900FBE0F90EA
:100330001F9018951F920F920FB60F920BB60F9247
:100340001124EF920F932F933F934F935F936F93EB
:100350007F938F939F93AF93BF93EF93FF93DF931D
:10036000CF9300D0CDB7DEB719821A828FE00E94FA
:100370008C04A89582FF07C086E00E948C048F71D0
:100380008093920D2AC183FF28C18091930D909193
:10039000940D019709F002C185E29DE06CE6AE0183
:1003A0004E5F5F4F9E012F5F3F4F0E940D058823D8
:1003B00009F413C18981882309F40FC12091420EE9
:1003C0003091430E4091440E5091450E8091250D81
:1003D0009091260DA091270DB091280D82179307BB
:1003E000A407B50709F088C08091A4009091A500EA
:1003F0009093210D8093200D1092A5001092A400DF
:100400008091220D882331F48CE390E090932302B5
:10041000809322028091220290912302E091470E64
:100420002091950D0A96F0E0B4E0EE0FFF1FBA950B
:10043000E1F7E20FF11DEC5DFD4F2081820F911D70
:100440009093A9008093A800A8950E949110009114
:10045000220DE090950D85E29DE06091920D409116
:10046000910D2A810E945413082F86E00E948C046B
:100470008F718093910D8430F8F40023E9F0E091BE
:10048000460E8091950DF0E0A4E0EE0FFF1FAA95B7
:10049000E1F7E80FF11DEC53FD4F82E060810E940F
:1004A000120480E293E00197F1F785E29DE0602F6E
:1004B00070E00E94090419C00E94FB03E091460EFF
:1004C0008091950DF0E074E0EE0FFF1F7A95E1F753
:1004D000E80FF11DEC53FD4F81E060810E94120492
:1004E00080E293E00197F1F7A8958091220D809327
:1004F000240D1092220D71C08091420E9091430EF6
:10050000A091440EB091450E0097A105B10509F0E8
:1005100064C08091920D853008F45FC0A8950E9458
:1005200091108091420E9091430EA091440EB09193
:10053000450E2091250D3091260D4091270D5091AB
:10054000280D82179307A407B50771F08091290D34
:100550008150823048F42093420E3093430E4093F2
:10056000440E5093450EA8950E94FB03E091460E61
:100570008091950DF0E064E0EE0FFF1F6A95E1F7C2
:10058000E80FF11DEC53FD4F81E060810E941204E1
:1005900080E293E00197F1F7A8951FC00E94FB034A
:1005A000E091460E8091950DF0E054E0EE0FFF1FB4
:1005B0005A95E1F7E80FF11DEC53FD4F81E06081A2
:1005C0000E94120480E293E00197F1F7A89586E07B
:1005D0000E948C048F718093910D0F900F90CF919A
:1005E000DF91FF91EF91BF91AF919F918F917F919B
:1005F0006F915F914F913F912F910F91EF900F90DD
:100600000BBE0F900FBE0F901F901895DF93CF93E6
:1006100000D000D0CDB7DEB789E492E0A0E0B0E032
:1006200089839A83AB83BC83CE01019660E070E03E
:1006300044E050E00E94402482E49EE064E070E0E8
:1006400042E550E00E9440240F900F900F900F90D1
:10065000CF91DF910895EF92FF920F93DF93CF93A5
:10066000CDB7DEB768970FB6F894DEBF0FBECDBF2B
:1006700019821A821B821C820E94B300CE0101964D
:1006800060E070E044E050E00E94302489819A816B
:10069000AB81BC8105E0E02EF12CEC0EFD1E8954EF
:1006A0009240A040B040D1F482E49EE064E070E06B
:1006B00042E550E00E94302480E092E00E946B0806
:1006C0002091420E3091430E4091440E5091450EC0
:1006D000C701B90140E020E001E018C080E192E0EC
:1006E0000E946B0869817A81C70140E020E001E047
:1006F0000E94F806C7010E946B0880E292E00E9407
:100700006B08C70169E472E040E020E00E94F8064F
:10071000C7010E946B088DE092E00E946B0868960A
:100720000FB6F894DEBF0FBECDBFCF91DF910F9112
:10073000FF90EF9008958AEF90E0909323028093CA
:1007400022020E942B038091460E8A3010F480937F
:10075000460E0E9437040E94FB03E091460E8091F2
:10076000950DF0E094E0EE0FFF1F9A95E1F7E80F8A
:10077000F11DEC53FD4F81E060810E94120485E081
:100780006FE040E020E00E94B0040E94D603109287
:10079000A5001092A40080912202909123029093D0
:1007A000A9008093A8000E94911008951092A500BE
:1007B0001092A4001092A00085E08093A1008FEF1A
:1007C00090E09093A9008093A800E2E7F0E0808198
:1007D000826080837894089594B7977F94BFE0E611
:1007E000F0E090819861908387708860808384B7FF
:1007F000877F84BF08958091950D8F3030F480916C
:10080000950D8F5F8093950D02C01092950D80E03D
:1008100008959C01862FB9010E9465052C9A2C9899
:1008200080E008951F93182F262F88E06FE140E0A5
:100830000E94B004812F90E09093940D8093930DCB
:10084000113019F482E066E008C085E060E847E016
:1008500021E00E94B00482E069E00E947D048EE005
:100860006CE00E947D04789480E01F9108950F93BE
:100870001F9384E00E9458040CEF13E0C801019715
:10088000F1F717982C988CE090E00197F1F7179A00
:1008900082E068E00E947D04C8010197F1F781E0E1
:1008A0006FE140E00E949D0480E01F910F91089548
:1008B0000F9A249A95B1936095B994B1976094B9C1
:1008C000239890E59CBD9CB59C7F9CBD9DB59E7F6B
:1008D0009DBD2CB5982F9370922B9CBD9DB5869590
:1008E00086958170982B9DBDEAE6F0E080818C6052
:1008F000808380E28CBBED9A0895806C9FB7F8945A
:1009000028988EBD0DB407FEFDCF6EBD0DB407FE59
:10091000FDCF289A9FBF08958F7380689FB7F89482
:1009200028988EBD0DB407FEFDCF8EBD0DB407FE19
:10093000FDCF8EB5289A9FBF0895FF920F931F9306
:10094000062FF42E0E948C04082310E002C0159597
:100950000795FA94E2F7802F1F910F91FF90089569
:10096000DF92EF92FF920F931F93D82EF62EE42E74
:10097000022F0E948C046F2D6095682310E002C046
:10098000000F111FEA94E2F7F0226F298D2D0E94CB
:100990007D041F910F91FF90EF90DF900895CB01A0
:1009A0000895FC01DA015FB7F894289880E28EBDC3
:1009B0000DB407FEFDCF1EBC0DB407FEFDCF4EB536
:1009C000641730F1942F20E030E01EBC0DB407FE18
:1009D000FDCF8EB52827022E2295207F2025032EBD
:1009E000322F22952F700226269532272327220F99
:1009F000220F220F20258083915011F03196E5CFF0
:100A0000109739F01C92232B21F481E08C9301C0C4
:100A10004068289A5FBF842F0895FF920F931F9319
:100A2000CF93DF938C01EA01D901FFB6F89428989F
:100A300080E28EBD0DB407FEFDCF1EBC0DB407FED7
:100A4000FDCF9EB5691708F436C020E030E040E0E5
:100A500050E0692F70E01CC01EBC0DB407FEFDCF36
:100A60008EB5F801E20FF31F80834827042E4295CC
:100A7000407F4025052E542F42954F700426469501
:100A800054274527440F440F440F40252F5F3F4F05
:100A90002617370708F3109729F01C92452B11F4FD
:100AA00081E08C93209741F01EBC0DB407FEFDCF72
:100AB0008EB5888301C09068289AFFBE892FDF9188
:100AC000CF911F910F91FF900895982FFB012FB7A1
:100AD000F894289880E68EBD0DB407FEFDCF9EBD2C
:100AE0000DB407FEFDCF80818EBD915011F031967F
:100AF000F7CF0DB407FEFDCF289A2FBF0895FC0154
:100B0000DA013FB7F894289880E28EBD0DB407FE55
:100B1000FDCF1EBC0DB407FEFDCF2EB56217A0F0B1
:100B2000922F1EBC0DB407FEFDCF8EB58083915071
:100B300011F03196F6CF109741F01EBC0DB407FEB0
:100B4000FDCF8EB58C9301C02068289A3FBF822FBD
:100B50000895833309F080E0089583E30895E82F32
:100B6000F0E0EE0FFF1FE656F14F20813181C90101
:100B70000895E82FF0E0EE0FFF1FE656F14F1182C7
:100B8000108208959B01AC01529A53985A9A5B9A2D
:100B900064E0220F331F441F551F6A95D1F760E0B0
:100BA00072E18AE790E00E94802321503040109249
:100BB000CD002093CC0080E48093C80088E9809326
:100BC000C90086E08093CA00789408959B01AC0127
:100BD000689A6998709A719A74E0220F331F441FC3
:100BE000551F7A95D1F760E072E18AE790E00E94A4
:100BF0008023215030401092C5002093C40080E42F
:100C00008093C00088E98093C10086E08093C20091
:100C100078940895FC018091970E8823D1F4F09385
:100C2000990EE093980E6093970E20919C0E309150
:100C30009D0E808190E08227932790939D0E809354
:100C40009C0E80818093CE008091C9008062809349
:100C5000C9008091970E8823E1F70895FC018091E7
:100C6000940E8823D1F4F093960EE093950E609342
:100C7000940E20919A0E30919B0E808190E08227F5
:100C8000932790939B0E80939A0E80818093C60049
:100C90008091C10080628093C1008091940E88236E
:100CA000E1F70895DF93CF930F92CDB7DEB7898335
:100CB000CE01019661E00E942E060F90CF91DF9148
:100CC0000895DF93CF930F92CDB7DEB78983CE011E
:100CD000019661E00E940A060F90CF91DF9108957E
:100CE0001F920F920FB60F920BB60F9211242F93F3
:100CF0003F938F939F93EF93FF93E091980EF09122
:100D0000990E3196F093990EE093980E3197809159
:100D1000970E81508093970E8091970E882391F0C3
:100D200080919C0E90919D0E2181332727FD309557
:100D30002827392730939D0E20939C0E8181809324
:100D4000CE0005C08091C9008F7D8093C900FF91BE
:100D5000EF919F918F913F912F910F900BBE0F902C
:100D60000FBE0F901F9018951F920F920FB60F9203
:100D70000BB60F9211242F933F938F939F93EF9372
:100D8000FF93E091950EF091960E3196F093960EAA
:100D9000E093950E31978091940E81508093940E3C
:100DA0008091940E882391F080919A0E90919B0EE1
:100DB0002181332727FD30952827392730939B0E33
:100DC00020939A0E81818093C60005C08091C10056
:100DD0008F7D8093C100FF91EF919F918F913F9103
:100DE0002F910F900BBE0F900FBE0F901F90189574
:100DF000BF92CF92DF92EF92FF920F931F93DF93F8
:100E0000CF93CDB7DEB72C970FB6F894DEBF0FBEE9
:100E1000CDBF6C01FB01B42EE22E77FD02C0FF2492
:100E200008C0F095E195FF4F8DE2D6018C93FF2429
:100E3000F39440E08E010F5F1F4F10C0200F311F51
:100E4000CF016AE070E00E946D23805DD9018C9330
:100E5000CF016AE070E00E946D23FB01242F30E097
:100E60004F5FEA30F10554F7020F131F8E2F805D9C
:100E7000F8018083642FCE01019620E305C0FC01B8
:100E8000E60FF11D20836F5FE616C8F76B15B8F308
:100E9000862F90E09E012F5F3F4FF901E80FF91F69
:100EA00010820197D901A80FB91F019640E050E0C8
:100EB0008C012E2D30E07EE214C0C801841B950BFE
:100EC0008217930729F4F601EF0DF11D7083F39457
:100ED000F601EF0DF11D8C918083F3944F5F5F4F0E
:100EE0001197461750F3F601EF0DF11D1082C60160
:100EF0002C960FB6F894DEBF0FBECDBFCF91DF9119
:100F00001F910F91FF90EF90DF90CF90BF900895C9
:100F10004F925F926F927F928F929F92AF92BF9209
:100F2000CF92DF92EF92FF920F931F93DF93CF93B5
:100F3000CDB7DEB72C970FB6F894DEBF0FBECDBF8E
:100F40003C016A017B01422E502E77FD02C099249C
:100F50000DC0F094E094D094C094C11CD11CE11C4D
:100F6000F11C8DE2F30180839924939488245E011F
:100F70000894A11CB11C19C00A0D1B1DC701B601A4
:100F80002AE030E040E050E00E94A223605DF801DA
:100F90006083C701B6012AE030E040E050E00E94E3
:100FA000A223C901DA016C017D01082D10E08394B0
:100FB000FAE0CF16D104E104F104F4F6A00EB11E5C
:100FC0008C2D805DF5018083482DCE01019620E3B4
:100FD00005C0FC01E40FF11D20834F5F5416C8F7D4
:100FE0004415B8F3842F90E09E012F5F3F4FF90125
:100FF000E80FF91F10820197D901A80FB91F0196B8
:1010000020E030E0BC01052D10E05EE214C0CB0111
:10101000821B930B8017910729F4F301E90DF11D51
:1010200050839394F301E90DF11D8C918083939487
:101030002F5F3F4F1197241750F3F301E90DF11D76
:101040001082C3012C960FB6F894DEBF0FBECDBF41
:10105000CF91DF911F910F91FF90EF90DF90CF9094
:10106000BF90AF909F908F907F906F905F904F90C8
:101070000895DC010D900020E9F71197A81BB90B2A
:101080006A2F0E942E060895EF92FF920F93DF932E
:10109000CF93CDB7DEB72A970FB6F894DEBF0FBE59
:1010A000CDBFBC017E010894E11CF11CC70140E0EA
:1010B00020E001E00E94F806C7010E9439082A9644
:1010C0000FB6F894DEBF0FBECDBFCF91DF910F9169
:1010D000FF90EF900895DC010D900020E9F7119743
:1010E000A81BB90B6A2F0E940A060895CF92DF92BF
:1010F000EF920F93DF93CF93CDB7DEB72A970FB65A
:10110000F894DEBF0FBECDBFAB01BC016E010894E9
:10111000C11CD11CC60120E000E0EE24E3940E9433
:101120008807C6010E946B082A960FB6F894DEBFA6
:101130000FBECDBFCF91DF910F91EF90DF90CF9099
:101140000895EF92FF920F93DF93CF93CDB7DEB761
:101150002A970FB6F894DEBF0FBECDBFBC017E014B
:101160000894E11CF11CC70140E020E001E00E946E
:10117000F806C7010E946B082A960FB6F894DEBFE6
:101180000FBECDBFCF91DF910F91FF90EF900895EB
:10119000809881988298839886E880937A0080E48A
:1011A00080937C000895806480937C0086E880931F
:1011B0007A0080917A00806480937A0080917A002E
:1011C00084FFFCCF2091780030917900C901089507
:1011D000E82F8091840E8E1709F43FC080918A0E0B
:1011E0008E17D9F180917E0E813118F080E18093C5
:1011F0007E0E20917F0E3091800E8091810E909115
:10120000820E4FEF5FE1DA01A81BB90BA217B307FB
:1012100050F48091810E9091820E481B590B50938F
:10122000800E40937F0E8091810E9091820E23E07C
:10123000880F991F2A95E1F79093650380936403C3
:1012400080917E0EE81748F4F0E06052714DEE0F89
:10125000FF1FE556F24F7183608308951092850059
:1012600010928400089580E090E020EE3EE2FC01C0
:10127000EE0FFF1FE556F24F318320830196803138
:101280009105A9F7259A2D9A82E08093800088E144
:10129000809381008091800080688093800080919D
:1012A00081008160809381008FEF9FEF9093870092
:1012B0008093860080916F00816080936F007894A6
:1012C00008951F920F920FB60F920BB60F92112432
:1012D0002F933F934F935F938F939F93EF93FF933E
:1012E0008091830E882371F4809188009091890009
:1012F0002091640330916503820F931F90938700C0
:10130000809386005091980D80917E0E581708F0BA
:101310008CC08091840E851791F5E091870EF09135
:10132000880E43E0EE0FFF1F4A95E1F74091990DBB
:101330008091850E481780F48091890EE42FF0E0AB
:10134000E80FF11DEE0FFF1FE256F14F0190F08103
:10135000E02DE052F14D0CC08091860E823061F498
:101360008091850E90E0242F30E08217930724F0BF
:101370004F5F4093990D38C01092990D35C0809100
:101380008A0E8517E1F5E0918D0EF0918E0E23E027
:10139000EE0FFF1F2A95E1F740919A0D80918B0E79
:1013A000481780F480918F0EE42FF0E0E80FF11DD4
:1013B000EE0FFF1FE256F14F0190F081E02DE05259
:1013C000F14D0CC080918C0E823061F480918B0EB7
:1013D00090E0242F30E08217930724F04F5F409372
:1013E0009A0D02C010929A0D80916403909165034A
:1013F000E81BF90BF093970DE093960D12C0E52FC3
:10140000F0E0EE0FFF1FE556F24F808191812091B1
:10141000640330916503821B930B9093970D809327
:10142000960D5F5F5093980D0FC080917F0E909145
:10143000800E53E0880F991F5A95E1F79093970D0E
:101440008093960D1092980D8091830E2091960DA9
:101450003091970D882329F43093890020938800D8
:1014600012C08091880090918900820F931F909301
:101470008700809386008091640390916503909328
:10148000890080938800FF91EF919F918F915F91E8
:101490004F913F912F910F900BBE0F900FBE0F9069
:1014A0001F901895519A509A599A589AE9EBF0E082
:1014B00080818360808380E28093B80084E08093A1
:1014C000BC00089584EA8093BC00089584E9809369
:1014D000BC00089520E030E002C02F5F3F4F8091B4
:1014E000BC0087FD06C083E228323807B1F780E0F0
:1014F000089580E02852334208F481E008958093F3
:10150000BB0084E88093BC000895813029F4809169
:10151000BC008F70806C04C08091BC008F708068AC
:101520008093BC0008958091BB0008958091B9001C
:101530000895EF92FF920F931F93CF93DF93182F8D
:10154000E62E042FF52E84EA8093BC000E946A0ADE
:101550001093BB0084E88093BC000E946A0A8091CB
:10156000B9008871B1F4802F9F2D9C01E90110E032
:1015700004E808C089918093BB000093BC000E94DE
:101580006A0A1F5F1E15B0F384E98093BC0081E0F6
:1015900004C084E98093BC0080E0DF91CF911F916B
:1015A0000F91FF90EF9008950F931F93182F062F20
:1015B00084EA8093BC000E946A0A1093BB0014E87E
:1015C0001093BC000E946A0A8091B900887159F09A
:1015D0000093BB001093BC000E946A0A84E98093C8
:1015E000BC0081E004C084E98093BC0080E01F91CE
:1015F0000F910895FF920F931F93182F062FF42E2B
:1016000084EA8093BC000E946A0A1093BB0014E82D
:101610001093BC000E946A0A8091B900887189F019
:101620000093BB001093BC000E946A0AF092BB00BA
:101630001093BC000E946A0A84E98093BC0081E098
:1016400004C084E98093BC0080E01F910F91FF905B
:101650000895CF92DF92EF92FF921F93CF93DF9383
:10166000182FF62E6A0184EA8093BC000E946A0A51
:101670001F5F1093BB0084E88093BC000E946A0A3D
:101680008091B900887159F510E0CF2DD0E02197F5
:101690000CC081E00E94850A0E946A0A8091BB000A
:1016A000F70180830E946A0A1F5F812F90E0760114
:1016B000E80EF91E8C179D0764F380E00E94850AEE
:1016C0000E946A0A8091BB00F70180830E946A0A27
:1016D00084E98093BC000E946A0A81E006C084E924
:1016E0008093BC000E946A0A80E0DF91CF911F9135
:1016F000FF90EF90DF90CF9008950F931F93DF93AB
:10170000CF9300D0CDB7DEB781E489831A8282E41B
:1017100061E08E010F5F1F4FA8010E94990A81307E
:1017200011F080E006C082E462E0A8010E94290B6B
:1017300081E00F900F90CF91DF911F910F9108954D
:101740000F931F93DF93CF9300D0CDB7DEB781E423
:1017500089831A8282E461E08E010F5F1F4FA80126
:101760000E94990A813029F482E462E0A8010E9473
:10177000290B998180E02A8130E0282B392BC9017F
:101780000F900F90CF91DF911F910F9108952F929D
:101790003F924F925F926F927F928F929F92AF9201
:1017A000BF92CF92DF92EF92FF920F931F93DF933E
:1017B000CF93CDB7DEB72E970FB6F894DEBF0FBE2E
:1017C000CDBFFE0131968AE0DF011D928A95E9F7CF
:1017D0008EEE64EF4EE20E94FA0A813009F588E04D
:1017E00092E028EC30E0F9013197F1F70197D9F751
:1017F0008EEE66EF0E94D40A813079F48EEE62E0BC
:10180000AE014F5F5F4F0E94290B998180E02A81D2
:10181000022F10E0082B192B09C086E693E002C0C6
:101820008DE693E00E946B0800E010E08EEE64EF1E
:1018300044EF0E94FA0A8130D1F588E29AE028EC60
:1018400030E0F9013197F1F70197D9F78EEE66EFA5
:101850000E94D40A813041F58EEE63E0AE014F5F05
:101860005F4F0E94290B898190E0A0E0B0E02C013D
:10187000332422248B8190E0A0E0B0E0282A392A8A
:101880004A2A5B2A9A8180E0AA2797FDA095BA2F61
:10189000282A392A4A2A5B2A45E0559447943794E6
:1018A00027944A95D1F70AC084E793E002C08BE7FA
:1018B00093E00E946B08222433242101B801882779
:1018C00077FD8095982F2091CB0D3091CC0D40E085
:1018D00050E0621B730B840B950B2091C90D309166
:1018E000CA0D40E050E00E943A237B018C013FE0AA
:1018F00015950795F794E7943A95D1F76091D30D34
:101900007091D40D882777FD8095982F2BE0660F76
:10191000771F881F991F2A95D1F72091D50D3091F7
:10192000D60D442737FD4095542F2E0D3F1D401FE7
:10193000511F0E94A22359016A01AE0CBF1CC01E98
:10194000D11E88E090E0A0E0B0E0A80EB91ECA1E4B
:10195000DB1ED601C50114E0B595A795979587952F
:101960001A95D1F79093BC0D8093BB0D88E590EF4D
:10197000AFEFBFEFA80EB91ECA1EDB1EC601B50130
:10198000A60195010E943A233B014C01ACE09594DD
:10199000879477946794AA95D1F72091C50D3091DB
:1019A000C60D442737FD4095542FC601B5010E944E
:1019B0003A237B018C01FDE015950795F794E79498
:1019C000FA95D1F782E090E0A0E0B0E0E80EF91ED1
:1019D0000A1F1B1F2091CD0D3091CE0D442737FDDE
:1019E0004095542FC401B3010E943A23BC019927AA
:1019F00077FD9095892FE60EF71E081F191F52E0FC
:101A000015950795F794E7945A95D1F780E090E8FB
:101A1000A0E0B0E0E80EF91E0A1F1B1F2091C70DC1
:101A20003091C80D40E050E0C801B7010E943A2350
:101A3000DC01CB014FE0B695A795979587954A9520
:101A4000D1F78B879C87AD87BE872091C30D3091DE
:101A5000C40D442737FD4095542FC601B5010E949F
:101A60003A237B018C013BE015950795F794E794A9
:101A70003A95D1F78091C10D9091C20DAA2797FD9B
:101A8000A095BA2F22E0880F991FAA1FBB1F2A9585
:101A9000D1F7E80EF91E0A1F1B1F2091CF0D3091C0
:101AA000D00D442737FD4095542FC401B3010E9447
:101AB0003A23ABE09595879577956795AA95D1F7E9
:101AC000E60EF71E081F191FEE0CFF1C001F111F4A
:101AD0002E183F08400A510AC201B1012AE638E136
:101AE00040E050E00E943A2397FD0FC0660F771F39
:101AF000881F991F2B853C854D855E850E9480231C
:101B0000C901DA015C016D010CC02B853C854D8556
:101B10005E850E94802359016A01AA0CBB1CCC1C63
:101B2000DD1C5527D7FC5A954D2D3C2D2B2DCA0178
:101B3000B9010E943A232EED3BE040E050E00E94C4
:101B40003A237B018C01C601B50123E433EE4FEF4C
:101B50005FEF0E943A23BC01992777FD9095892F6A
:101B60006153714F8F4F9F4F78011127F7FC1095EC
:101B7000012F6E0D7F1D801F911F24E09595879585
:101B8000779567952A95D1F76A0D7B1D8C1D9D1D54
:101B90006093BD0D7093BE0D8093BF0D9093C00DEB
:101BA00081E02E960FB6F894DEBF0FBECDBFCF9169
:101BB000DF911F910F91FF90EF90DF90CF90BF903A
:101BC000AF909F908F907F906F905F904F903F90DD
:101BD0002F90089582E893E00E946B088091BB0DDE
:101BE0009091BC0D6AE070E00E946D23882777FD1C
:101BF0008095982F0E94760889E893E00E946B08F0
:101C00008091BB0D9091BC0D6AE070E00E946D2345
:101C1000AA2797FDA095BA2FBC01CD010E94760896
:101C20008BE893E00E946B088091BB0D9091BC0DF6
:101C300008958EE893E00E946B086091BD0D70914D
:101C4000BE0D8091BF0D9091C00D0E9476088BE86B
:101C500093E00E946B086091BD0D7091BE0D809164
:101C6000BF0D9091C00D08950F931F93DF93CF93F5
:101C7000CDB7DEB72A970FB6F894DEBF0FBECDBF43
:101C80008E010F5F1F4F8AE0F80111928A95E9F7E4
:101C90008EEE64EF4EE20E94FA0A813011F080E08D
:101CA000DAC18EEE6AEA0E94D40A8EEE62E0A801E2
:101CB0000E94290B813081F4898190E0A0E0B0E09E
:101CC000BA2FA92F982F88272A8130E0282B392B6B
:101CD0003093C20D2093C10D8EEE6CEA0E94D40A9F
:101CE0008EEE62E0AE014F5F5F4F0E94290B8130A4
:101CF00081F4898190E0A0E0B0E0BA2FA92F982F5D
:101D000088272A8130E0282B392B3093C40D20936B
:101D1000C30D8EEE6EEA0E94D40A8EEE62E0AE0132
:101D20004F5F5F4F0E94290B813081F4898190E0E1
:101D3000A0E0B0E0BA2FA92F982F88272A8130E0A1
:101D4000282B392B3093C60D2093C50D8EEE60EBFA
:101D50000E94D40A8EEE62E0AE014F5F5F4F0E9498
:101D6000290B813081F4898190E0A0E0B0E0BA2FA6
:101D7000A92F982F88272A8130E0282B392B3093E0
:101D8000C80D2093C70D8EEE62EB0E94D40A8EEE32
:101D900062E0AE014F5F5F4F0E94290B813081F4FA
:101DA000898190E0A0E0B0E0BA2FA92F982F882772
:101DB0002A8130E0282B392B3093CA0D2093C90D8E
:101DC0008EEE64EB0E94D40A8EEE62E0AE014F5FAD
:101DD0005F4F0E94290B813081F4898190E0A0E05F
:101DE000B0E0BA2FA92F982F88272A8130E0282B1E
:101DF000392B3093CC0D2093CB0D8EEE66EB0E94E9
:101E0000D40A8EEE62E0AE014F5F5F4F0E94290B55
:101E1000813081F4898190E0A0E0B0E0BA2FA92F51
:101E2000982F88272A8130E0282B392B3093CE0D2C
:101E30002093CD0D8EEE68EB0E94D40A8EEE62E008
:101E4000AE014F5F5F4F0E94290B813081F4898181
:101E500090E0A0E0B0E0BA2FA92F982F88272A8120
:101E600030E0282B392B3093D00D2093CF0D8EEE00
:101E70006AEB0E94D40A8EEE62E0AE014F5F5F4FC4
:101E80000E94290B813081F4898190E0A0E0B0E0CC
:101E9000BA2FA92F982F88272A8130E0282B392B99
:101EA0003093D20D2093D10D8EEE6CEB0E94D40AAC
:101EB0008EEE62E0AE014F5F5F4F0E94290B8130D2
:101EC00081F4898190E0A0E0B0E0BA2FA92F982F8B
:101ED00088272A8130E0282B392B3093D40D20938A
:101EE000D30D8EEE6EEB0E94D40A8EEE62E0AE0150
:101EF0004F5F5F4F0E94290B813081F4898190E010
:101F0000A0E0B0E0BA2FA92F982F88272A8130E0CF
:101F1000282B392B3093D60D2093D50D85E993E0EE
:101F20000E946B086091C10D7091C20D882777FDEA
:101F30008095982F0E9476088CE993E00E946B08A8
:101F40006091C30D7091C40D882777FD8095982FFF
:101F50000E9476088CE993E00E946B086091C50DA1
:101F60007091C60D882777FD8095982F0E9476087E
:101F70008CE993E00E946B086091C70D7091C80DC9
:101F800080E090E00E9476088CE993E00E946B0864
:101F90006091C90D7091CA0D80E090E00E947608B2
:101FA0008CE993E00E946B086091CB0D7091CC0D91
:101FB00080E090E00E9476088CE993E00E946B0834
:101FC0006091CD0D7091CE0D882777FD8095982F6B
:101FD0000E9476088CE993E00E946B086091CF0D17
:101FE0007091D00D882777FD8095982F0E947608F4
:101FF0008CE993E00E946B086091D10D7091D20D35
:10200000882777FD8095982F0E9476088CE993E0C9
:102010000E946B086091D30D7091D40D882777FDD5
:102020008095982F0E9476088CE993E00E946B08B7
:102030006091D50D7091D60D882777FD8095982FEA
:102040000E9476088CE993E00E946B088BE893E08D
:102050000E946B0881E02A960FB6F894DEBF0FBE8F
:10206000CDBFCF91DF911F910F910895FC01808129
:10207000860F80830895FC01808181958083089577
:10208000FC018081860F80830895FC018081819509
:1020900080830895FC0180819181860F971F918331
:1020A00080830895FC0180819181909581959F4F57
:1020B000918380830895FC0180819181860F971F11
:1020C000918380830895FC01808191819095819511
:1020D0009F4F918380830895FC01882777FD809529
:1020E000982F2081318142815381260F371F481F4D
:1020F000591F20833183428353830895FC018081DB
:102100009181A281B381B095A095909581959F4FC3
:10211000AF4FBF4F80839183A283B3830895279AE3
:1021200008952F9A08952F980895E42FF0E0DF0185
:10213000A25CBF4E1C92DF01A65DBF4E8C93EA5E8F
:10214000FF4E10826093F10D8091E70D8A3F28F4D5
:102150008091E70D8F5F8093E70D6623C1F080913A
:10216000EB0D9091EC0D66956695262F30E0820F71
:10217000931F9093EC0D8093EB0D8091ED0D90915A
:10218000EE0D280F391F3093EE0D2093ED0D809149
:10219000EB0D9091EC0D855F9140F0F02091ED0DED
:1021A0003091EE0D6091EB0D7091EC0D84E690E0B6
:1021B000AC01249FC001259F900D349F900D1124E8
:1021C0000E9459236093EA0D1092EC0D1092EB0DD2
:1021D0001092EE0D1092ED0D08951F920F920FB612
:1021E0000F920BB60F921124EF92FF920F931F9351
:1021F0002F933F934F935F936F937F938F939F930F
:10220000AF93BF93EF93FF939091C6009093EF0D20
:1022100080911D0E80931E0E80911C0E80931D0ECA
:1022200080911B0E80931C0E80911A0E80931B0EC2
:1022300090931A0E8091190E882349F4943209F074
:102240000CC181E08093190E1092180E06C18130E6
:1022500009F041C02091180E253031F58091040E0F
:10226000823551F48091050E8D3401F58091060E72
:102270008334E1F482E00BC08734C1F48091050E11
:10228000873451F48091060E813481F483E0809389
:10229000190E1092180E1AC0833541F48091060E63
:1022A000813421F484E0F3CF243170F4E22FF0E0A4
:1022B000EE5FF14F9083E22FEF5FE093180EF0E0B6
:1022C000EE5FF14F108202C01092190E1092170E9D
:1022D0001092160EC2C08230E1F59D3009F4BBC0E9
:1022E0009C3209F0A9C0F090160E83E18F1508F416
:1022F000A3C0E090170EE4E0EE1639F0F6E0EF161A
:1023000021F082E0E81609F091C00F2D10E082E084
:102310009EE00E94F823000F111F06581F4EF8017F
:1023200091838083F394F092160EE2E0FEE090E059
:1023300080818E3249F40F2D10E0892F90E08D5F5F
:10234000914F0E94F82367C09F5F3196943181F7C7
:102350006DC0833009F047C09D3009F47CC09C32C9
:1023600009F06AC0F090160EF3E1FF1508F464C09E
:10237000E090170E85E0E81608F458C0E6E0EE1588
:1023800020F4F8E0EF1609F051C00F2D10E00A5FBD
:102390001F4F82E09EE00E94F8239C01000F111F56
:1023A00006581F4EF80131832083F394F092160EE5
:1023B00020E030E0822FF901EE5FF14FE081EE2363
:1023C000A9F1EE3251F40F2D10E00A5F1F4F90E09B
:1023D0008D5F914F0E94F8231EC02F5F3F4F243125
:1023E000310541F723C08430B1F59D30A1F19C3215
:1023F00019F5F090160EF3E1FF15F0F0E090170ECE
:1024000081E0E81699F40F2D10E0065F1F4F82E07F
:102410009EE00E94F8239C01000F111F06581F4EDA
:10242000F80131832083F394F092160E1092180E67
:10243000E394E092170E11C0A091180EEA2FF0E07D
:10244000EE5FF14F9083AF5FA093180EB0E0AE5FE8
:10245000B14F1C9202C01092190EFF91EF91BF91E3
:10246000AF919F918F917F916F915F914F913F912C
:102470002F911F910F91FF90EF900F900BBE0F9037
:102480000FBE0F901F9018951F920F920FB60F92CC
:102490000BB60F9211242F933F934F935F936F933B
:1024A0007F938F939F93AF93BF93EF93FF93DF93AC
:1024B000CF9300D000D000D0CDB7DEB75091CE0082
:1024C0005093F00D9091000E9093010E2091FF0D0E
:1024D0002093000E3091FE0D3093FF0D4091FD0DC5
:1024E0004093FE0D5093FD0D8091FA0D823001F561
:1024F0008091FC0D813309F08DC099832A833B8341
:102500004C835D831E82CE0101960E94F42320E05D
:1025100030E040E251E40E9416200E94401E611506
:10252000710509F475C070937D1060937C1070C0C4
:102530008091FA0D813009F073C08091FC0D8231D9
:1025400091F499832A833B834C831D821E82CE01A2
:1025500001960E94F823009709F45CC090937B10C9
:1025600080937A1057C0873191F499832A833B83F3
:102570004C831D821E82CE0101960E94F823009793
:1025800009F448C090937D1080937C1043C08F3134
:1025900089F499832A833B834C835D831E82CE0119
:1025A00001960E94F8230097A9F190937F108093E1
:1025B0007E1030C0843289F499832A833B834C8314
:1025C0005D831E82CE0101960E94F823009711F1CF
:1025D00090938110809380101DC08B32D9F4998321
:1025E0002A833B834C835D831E82CE0101960E9429
:1025F000F42320E030E048EC52E40E9416200E94D0
:10260000401E6115710521F0709383106093821054
:102610001092FA0D8091FC0D8F5F8093FC0D2CC001
:102620009734B9F42035A9F4323541F44D3489F4A6
:10263000533479F41092FC0D81E009C0373449F429
:10264000473439F4513429F41092FC0D82E0809320
:10265000FA0D8091000E823B79F48091FF0D853A4E
:1026600059F48091FE0D853639F45B3429F4F894E1
:1026700080E00E94EC03FFCF2696DEBFCDBFCF9156
:10268000DF91FF91EF91BF91AF919F918F917F91DA
:102690006F915F914F913F912F910F900BBE0F90D3
:1026A0000FBE0F901F901895EF920F93CF93DF936B
:1026B000EC01EE2DF0E0DF01A25CBF4E6C93DF0178
:1026C000A65DBF4E4C93EA5EFF4E20830093F10D52
:1026D00088819981AA81BB818093F30D9093F40D39
:1026E000A093F50DB093F60D1092E70D8091EB0DD0
:1026F0009091EC0D01969093EC0D8093EB0D0023DF
:10270000C1F08091EB0D9091EC0D202F2695269530
:1027100030E0820F931F9093EC0D8093EB0D80912E
:10272000ED0D9091EE0D280F391F3093EE0D209393
:10273000ED0D8091EB0D9091EC0D855F9140F0F0E7
:102740002091ED0D3091EE0D6091EB0D7091EC0D3F
:1027500084E690E0AC01249FC001259F900D349F3A
:10276000900D11240E9459236093EA0D1092EC0DF4
:102770001092EB0D1092EE0D1092ED0D8C818130C8
:1027800009F07DC088E08093E90D888D998D909344
:10279000210E8093200EE0E010C0F0E0DF011496DF
:1027A000AA0FBB1FAC0FBD1F8D919C91EE0FFF1F99
:1027B000EE5AFF4E91838083E22F8091E90D2E2FF8
:1027C0002F5FE81750F3E0931F0E8E818F3F39F48F
:1027D0008F81882321F08093130D1092E80D1092C1
:1027E0001F0E24C0842F90E0FC01EE0FFF1FDF01BD
:1027F000AE5ABF4E2D913C91E256F14F318320836A
:102800008E5B914FDC015896EC91F0E0EE0FFF1FCC
:10281000EE5AFF4E60817181660F771F842F0E94F0
:10282000E80880911F0E8F5F80931F0E40911F0E4E
:102830008091E90D4817B0F28E818093DD0D8E8175
:10284000E82FF0E08091E90D9F01280F311D203421
:1028500031058CF48091E90DE80FF11D8F8124E1A1
:10286000829FC00111248C5E9940EE0FFF1FE2563B
:10287000F14F9183808381E08093FB0D7CC0823097
:1028800009F079C080E18093E90D88A599A590931E
:10289000210E8093200EE0E010C0F0E0DF011496DE
:1028A000AA0FBB1FAC0FBD1F8D919C91EE0FFF1F98
:1028B000EE5AFF4E91838083E22F8091E90D2E2FF7
:1028C0002F5FE81750F3E0931F0E8E818F3F39F48E
:1028D0008F81882321F08093130D1092E80D1092C0
:1028E0001F0E24C0842F90E0FC01EE0FFF1FDF01BC
:1028F000AE5ABF4E2D913C91E256F14F3183208369
:102900008E5B914FDC015896EC91F0E0EE0FFF1FCB
:10291000EE5AFF4E60817181660F771F842F0E94EF
:10292000E80880911F0E8F5F80931F0E40911F0E4D
:102930008091E90D4817B0F28E818093DD0D8E8174
:10294000E82FF0E08091E90D9F01280F311D203420
:1029500031058CF48091E90DE80FF11D8F8124E1A0
:10296000829FC00111248C5E9940EE0FFF1FE2563A
:10297000F14F918380838091200E8093F20D80919E
:10298000DB0D8B3000F584E08C838091DB0D8D8333
:102990001E828091DB0D90E02AE130E0829FF00101
:1029A000839FF00D929FF00D1124E252F14F178A90
:1029B0006091DB0D8AE1689FB00111246252714F72
:1029C000CE0108960EC08091DB0D8C30F0F484E0CF
:1029D0008C838091DB0D8D831E82CE01089663EA85
:1029E00073E00E9421248091200E9091210E99A3E2
:1029F00088A301969093210E8093200E8091DB0D89
:102A00008F5F8093DB0D84E2B8C08091DB0D8F5F18
:102A10008093DB0D8150853110F01092DB0D83E047
:102A20008C838091140D8D838091200E9091210EC6
:102A30009987888701969093210E8093200E80912C
:102A4000140D813188F4893008F062C08330A1F11F
:102A5000843030F48130F1F0823009F084C01DC040
:102A6000843009F050C037C0833109F466C0843126
:102A700038F4813109F457C0823109F074C058C06C
:102A8000853109F464C0853108F45CC0863109F0F1
:102A90006AC062C00E831F826AC020E030E090E00E
:102AA00008C0E92FF0E0E25CFF4E8081280F311D65
:102AB0009F5F9031B0F31DC020E030E090E008C08F
:102AC000E92FF0E0E65DFF4E8081280F311D9F5F0A
:102AD0009031B0F30EC020E030E090E008C0E92F64
:102AE000F0E0EA5EFF4E8081280F311D9F5F90313C
:102AF000B0F390931F0E64E0369527956A95E1F741
:102B00003F832E8334C090E005970E94D30828C0ED
:102B1000E82FF0E0EE0FFF1FE85CF14F808191811C
:102B20008051984F1DC080917A1090917B1018C0F1
:102B300080917C1090917D1013C080917E109091B7
:102B40007F100EC0809180109091811009C08091FB
:102B500082109091831004C0809184109091851010
:102B60009F838E8304C08E831F821092140D8091E8
:102B7000140D8F5F8093140D8CE0DF91CF910F9136
:102B8000EF90089582EB93E00E946B080895CF9335
:102B9000DF9386EE93E00E946B08C0E0D0E08AEEFF
:102BA00093E00E946B08FE01E65DFF4E808190E09D
:102BB0000E94A1082196C031D10589F78CEE93E0DF
:102BC0000E946B08C0E0D0E08AEE93E00E946B08A0
:102BD000FE01E25CFF4E808190E00E94A1082196F8
:102BE000C031D10589F783EF93E00E946B08C0E004
:102BF000D0E08AEE93E00E946B08FE01EA5EFF4E91
:102C0000808190E00E94A1082196C031D10589F70A
:102C10008AEF93E00E946B088AEE93E00E946B08B3
:102C200080E090E00E94D3080E94A1088AEE93E021
:102C30000E946B0881E090E00E94D3080E94A108E6
:102C40008AEE93E00E946B0882E090E00E94D30835
:102C50000E94A1088AEE93E00E946B0883E090E056
:102C60000E94D3080E94A10881E094E00E946B08B2
:102C7000C0E0D0E08AEE93E00E946B08FE01EE0F08
:102C8000FF1FEE5AFF4E808191810E94A10821967C
:102C9000C031D10579F788E094E00E946B08C0E06C
:102CA000D0E08AEE93E00E946B08FE01EE0FFF1F5A
:102CB000E65BF14F808191810E94A1082196C83086
:102CC000D10579F78FE094E00E946B088091F10DB7
:102CD00090E00E94A1088AEE93E00E946B08809128
:102CE000ED0D9091EE0D0E94A1088AEE93E00E94F6
:102CF0006B088091EB0D9091EC0D0E94A1088AEE7B
:102D000093E00E946B088091EA0D90E00E94A10878
:102D10008AEE93E00E946B088091F30D9091F40D80
:102D2000A091F50DB091F60D0E94A1088AEE93E0F6
:102D30000E946B088091420E9091430EA091440E28
:102D4000B091450E0E94A1088AEE93E00E946B08A4
:102D50008091F20D90E00E94A10887E194E00E942A
:102D60006B08C0E0D0E08AEE93E00E946B08FE01A1
:102D7000EE0FFF1FE658FF4E808191810E94A1084F
:102D80002196CB30D10579F78EE194E00E946B0853
:102D9000DF91CF9108950F931F93CF93DF938FEF20
:102DA0000E9461068FEF0E94610640E050E020E043
:102DB00030E0F901E25CFF4E8081480F511D2F5F2A
:102DC0003F4F20313105A9F7A4E056954795AA95C4
:102DD000E1F7842F0E94610640E050E020E030E0FF
:102DE000F901EA5EFF4E8081480F511D2F5F3F4F72
:102DF00020313105A9F7F5E056954795FA95E1F7A9
:102E0000842F0E946106C0E0D0E08E01000F111FE8
:102E10000E5A1F4EF801808191818050984F892F62
:102E20000E946106F801808191810E9461062196CD
:102E3000C031D10551F7DF91CF911F910F910895C6
:102E4000CF93DF938FEF0E9461068FEF0E946106A0
:102E500040E050E020E030E0F901E25CFF4E80818C
:102E6000480F511D2F5F3F4F20313105A9F794E0E6
:102E7000569547959A95E1F7842F0E94610640E0A8
:102E800050E020E030E0F901EA5EFF4E8081480F1B
:102E9000511D2F5F3F4F20313105A9F785E0569531
:102EA00047958A95E1F7842F0E946106C0E0D0E043
:102EB000FE01EE0FFF1FEE5AFF4E80819181805080
:102EC000984F60E170E00E946D23862F0E9461069A
:102ED0002196C031D10561F7DF91CF9108950F930D
:102EE0001F93DF93CF9300D00F92CDB7DEB78BE166
:102EF00089838BE58A838AE48B838E010F5F1F4F62
:102F0000C80163E00E940A0682E089831A82C80130
:102F100062E00E940A060F900F900F90CF91DF9110
:102F20001F910F9108950F931F93DF93CF9300D0BC
:102F300000D0CDB7DEB78BE189838BE58A838BE345
:102F40008B8388E48C838E010F5F1F4FC80164E080
:102F50000E940A0682E089831A82C80162E00E9408
:102F60000A060F900F900F900F90CF91DF911F9155
:102F70000F9108951F93CF93DF930E946F170E94C4
:102F8000931782E294E00E946B088DE594E00E9422
:102F90006B088BE894E00E946B0883EC94E00E943D
:102FA0006B0882ED94E00E946B088091840E803162
:102FB00050F58BED94E00E946B088091850E90E0B7
:102FC0000E94A10883EE94E00E946B088091840E19
:102FD00090E001960E94A10884EF94E00E946B08A3
:102FE0008091860E90E00E94A10887EF94E00E94F5
:102FF0006B088091870E9091880E0E94A10889EF3E
:1030000094E00E946B088EEF94E00E946B088AE0C7
:1030100095E00E946B088CE195E00E946B088BE2C2
:1030200095E00E946B0881E395E00E946B0887E3BE
:1030300095E00E946B088DE395E00E946B088AE0A2
:1030400095E00E946B0881E595E00E946B08C0E066
:10305000D0E013E0FE01E25CFF4E8081819FC00161
:1030600011248B5590400E94A10880E695E00E94B3
:103070006B082196C031D10569F782E695E00E9480
:103080006B08C0E0D0E013E0FE01E65DFF4E8081FA
:10309000819FC00111248B5590400E94A10880E6B9
:1030A00095E00E946B082196C031D10569F782E84E
:1030B00095E00E946B08C0E0D0E013E0FE01E65D01
:1030C000FF4E4081FE01E25CFF4E8081819FC00186
:1030D000112450E09A01220F331F240F351F821B49
:1030E000930B0E94A10880E695E00E946B08219650
:1030F000C031D10519F782EA95E00E946B08C0E063
:10310000D0E0FE01EA5EFF4E808190E00E94A108BF
:1031100080E695E00E946B082196C031D10589F7C1
:1031200082EC95E00E946B088091F10D90E00E9486
:10313000A10882EE95E00E946B088091ED0D9091C0
:10314000EE0D0E94A10884EE95E00E946B0880912C
:10315000EB0D9091EC0D0E94A10886EE95E00E9487
:103160006B088091EA0D90E00E94A10888EE95E03E
:103170000E946B088091200D9091210D0E94A10862
:1031800084EE95E00E946B088091220290912302C8
:103190000E94A1088AE096E00E946B088091F30DDE
:1031A0009091F40DA091F50DB091F60D0E94A1083B
:1031B0008CE296E00E946B088091420E9091430E43
:1031C000A091440EB091450E0E94A1088FE296E0B6
:1031D0000E946B088091F20D90E00E94A10880E5AA
:1031E00096E00E946B088FE596E00E946B0880E0F5
:1031F00090E00E94D3080E94A10880E796E00E9418
:103200006B0881E090E00E94D3080E94A10884E747
:1032100096E00E946B0882E090E00E94D3080E9432
:10322000A10888E796E00E946B0883E090E00E9486
:10323000D3080E94A1088CE796E00E946B0883E8FF
:1032400096E00E946B088091660090E00E94A108C1
:1032500082E996E00E946B088CE996E00E946B0878
:103260008091460E90E00E94A1088BEA96E00E94B1
:103270006B088091470E90E00E94A10882E996E0D9
:103280000E946B088EEA96E00E946B0810E00FC067
:10329000E12FF0E0EE0FFF1FEE5AFF4E808191818B
:1032A0000E94A10880E695E00E946B081F5F809154
:1032B000E90D181768F382E996E00E946B088DEB20
:1032C00096E00E946B088091DD0D992787FD90950F
:1032D0000E94A10882E996E00E946B088CEC96E0BF
:1032E0000E946B0882EE95E00E946B088091890E27
:1032F00090E00E94A1088BED96E00E946B088091FF
:10330000890E2091850E90E0820F911D0E94A108E8
:103310008EED96E00E946B0810E011C08091890E3E
:10332000E80FF11DEE0FFF1FE256F14F80819181F2
:103330000E94A10880E695E00E946B081F5F8091C3
:10334000850E181750F4E12FF0E08091890E9F014F
:10335000280F311D203431050CF381EE96E00E94D8
:103360006B0882EE95E00E946B0880918F0E90E0D2
:103370000E94A1088BED96E00E946B0880918F0E51
:1033800020918B0E90E0820F911D0E94A1088EED7E
:1033900096E00E946B0810E011C080918F0EE80F3C
:1033A000F11DEE0FFF1FE256F14F808191810E94C7
:1033B000A10880E695E00E946B081F5F80918B0E4C
:1033C000181750F4E12FF0E080918F0E9F01280F25
:1033D000311D203431050CF382E996E00E946B0820
:1033E000DF91CF911F9108950F93FC010190002070
:1033F000E9F73197E81BF90BDB016D917C918E0F9A
:103400009F1F40E020E001E00E94F8060F91089520
:103410000F93FC0101900020E9F73197E81BF90BAD
:10342000DB016D917C918E0F9F1F40E020E001E059
:103430000E94F8060F9108950F93FC01019000205F
:10344000E9F73197E81BF90BDB016D917C918E0F49
:103450009F1F40E020E001E00E94F8060F910895D0
:103460000F93DC010D900020E9F71197A81BB90B11
:10347000FB016081772767FD70958A0F9B1F40E0F5
:1034800020E001E00E94F8060F9108950F93FC01DF
:1034900001900020E9F73197E81BF90BDB016C91F3
:1034A0008E0F9F1F70E040E020E001E00E94F806D0
:1034B0000F9108958F929F92AF92BF92CF92DF9219
:1034C000EF92FF920F931F93DF93CF93CDB7DEB7A9
:1034D000A0970FB6F894DEBF0FBECDBF282F19827C
:1034E0004091D80D9091D70DA92FB0E0FD01E35286
:1034F000F34FE081BE2EB40E8091900E882319F414
:1035000081E08093900E233309F46AC0243338F4A9
:10351000213309F4ACC0223309F0BCC013C02633F8
:1035200029F1283321F0243309F0B4C060C04423CA
:1035300011F0415012C0A851B34F8C91815080932B
:10354000D80D10C0242F30E0A851B34F8C9190E0DB
:1035500001972817390724F44F5F4093D80D02C014
:103560001092D80DB090D80DBE0E94C0AB2DB0E027
:10357000FD01EB54F84FE081E230F9F0E33030F434
:10358000EE23D9F0E13009F085C008C0E430F9F04D
:10359000E430E8F0E53009F07DC022C0AA0FBB1F7F
:1035A000AA50B84FED91FC9180819181A281B381A5
:1035B0008C509E4FAF4FBF4F4BC0AA0FBB1FAA509E
:1035C000B84FED91FC91808191810A9630C0AA0F8D
:1035D000BB1FAA50B84FED91FC9180818F5F45C011
:1035E0009A3010F49F5F46C01092D70D49C0AB2DA2
:1035F000B0E0FD01EB54F84FE081E23079F0E330C8
:1036000030F4EE2359F0E13009F044C013C0E43047
:1036100021F1E43010F1E530E9F529C0AA0FBB1F14
:10362000AA50B84FED91FC91808191810A979183C6
:10363000808330C0AA0FBB1FAA50B84FED91FC91F8
:1036400080819181A281B381845F9140A040B0408C
:1036500080839183A283B3831DC0AA0FBB1FAA508E
:10366000B84FED91FC9180818150808313C09923E4
:1036700021F091509093D70D03C08AE08093D70D2D
:103680001092D80DE091D70DF0E0E352F34FB080E7
:10369000B092D90D0B2D10E02091D90D8091900E94
:1036A00090E0820F911D0197081719074CF0809147
:1036B000900E2B2D281B822F8F5F8093D90D04C075
:1036C000B21610F4B092D90D89EF96E00E946B0803
:1036D000E091D70DF0E0E352F34F208181E090E0DC
:1036E000821B9109800F911F0E94A10884EE95E032
:1036F0000E946B08E091D70DF0E0E851F34F808114
:1037000090E00E94A1088DEF96E00E946B08E09186
:10371000D70DF0E0EE0FFF1FE953F34F8081918149
:103720000E946B088FEF96E00E946B0884E097E0A0
:103730000E946B08E091D70DF0E0EE0FFF1FE953F8
:10374000F34F6081718182EE9FE00E94212400E0AE
:1037500010E0C8018252914F66EE75E00E9421246C
:10376000065E1F4F31E00430130799F7A090D90D82
:103770007E010894E11CF11CEAE18E2E912C89C097
:103780001982BA1429F4C7016CE177E00E9416246B
:103790008601000F111FF801EE51F44F6081718115
:1037A000C7010E941624C7016EE177E00E9416242B
:1037B000F601EB54F84FE081E23001F1E33028F4F8
:1037C000EE2351F0E130C1F510C0E43039F1E430BE
:1037D000F0F0E53089F52BC00A50184FF8016081F0
:1037E0007181C7010E94081A27C00A50184FF801BA
:1037F00060817181C7010E94F4191EC00A50184FE0
:10380000F80160817181C7010E941C1A15C00A501D
:10381000184FF80160817181C7010CC00A50184F20
:10382000F80160817181C7010E94301A05C0C7018B
:1038300067ED7DE00E94461A80E297E00E946B08E7
:103840008091D90D9601281B3109C9010E94A10858
:103850008DEF96E00E946B08C7010E946B0884E21E
:1038600097E00E946B088091D90DF601E81BF109E1
:10387000EA30F1056CF4188EE89DC001E99D900DC9
:10388000F89D900D11248252914FB7010E9421247E
:10389000A394CA2CDD242091900E8091D90D90E044
:1038A000820F911DC816D906A4F430E43A1588F0A9
:1038B000E091D70DF0E0DF01A851B34F2C91E35216
:1038C000F34F808190E0820F911DC816D9060CF449
:1038D00057CF84E097E00E946B08A0960FB6F8944B
:1038E000DEBF0FBECDBFCF91DF911F910F91FF9033
:1038F000EF90DF90CF90BF90AF909F908F90089502
:10390000CF92DF92EF92FF920F931F93CF93DF93AB
:103910001092DA0D1092DC0D80E090E02AE130E0A8
:10392000829FF001839FF00D929FF00D1124E252CF
:10393000F14F108201968A30910591F7279A2F9ABC
:1039400080E090E0FC01EE0FFF1FEE5AFF4E118267
:103950001082019680319105A9F780E090E020E87F
:103960000FB6F89420936100809361000FBE399ADE
:10397000419A579A5F9A6B9A739804B603FC03C0F6
:1039800081E08093F90D1092F90D26982E9A60E04F
:1039900076E980E090E00E94C20587E297E00E940D
:1039A0006B0882EB93E00E946B0860E875E280E0B0
:1039B00090E00E94E6050E94520A0E94C8080E94F8
:1039C0009B030E94330980E00E945A1ACC24CA94B7
:1039D00001E093E0F92E84E0E82EC4ECD9E012E097
:1039E000D12E9091130DC092130D9F3F09F45AC030
:1039F0008091E80D882309F055C0992309F452C03D
:103A0000892F0E945A1A8091490E882309F1109239
:103A1000490E85E597E00E946B0820E030E0F9014F
:103A2000EE0FFF1FEE5AFF4E80819181F901EE0FDC
:103A3000FF1FE65BF14F918380832F5F3F4F28305C
:103A4000310569F70E9406038FE697E00E946B0834
:103A50008091930E8823C1F01092930E8DE797E02A
:103A60000E946B08F092840E1092890EE0928A0EEA
:103A700010928F0ED0937D0EC0937C0E0E94060391
:103A80008FE697E00E946B088091920E882341F0A8
:103A90001092920E0E9406038FE697E00E946B0838
:103AA0000093E80DA8958091F00D882371F4809122
:103AB000F70D813051F08091FB0D813009F0D7C0B6
:103AC0008091F80D853009F0D2C01091F00D109260
:103AD000F00D133619F4D092F80D04C0123429F405
:103AE000F092F80D0093F70D52C01D3619F41092A4
:103AF000F80DF8CF1636C1F420E030E0F901EE0FF2
:103B0000FF1FEE5AFF4E80819181F901EE0FFF1FDA
:103B1000E65BF14F918380832F5F3F4F2830310563
:103B200069F70E94060333C0133721F0812F8053B9
:103B30008A3028F40093F80D1092F70D28C0133541
:103B400029F40E94060382E997E01FC0123619F497
:103B50000E94AA001CC0153739F48091F70D902FF0
:103B6000981B9093F70D13C0123759F40E949317C6
:103B70008EE997E00E946B08F89480E00E94EC03C5
:103B8000FFCF193421F482EB93E00E946B088091FF
:103B9000F80D823009F463C0833030F4882359F083
:103BA000813009F064C00AC0833009F45BC08430FE
:103BB00009F05DC05AC00E94BA1759C0812F0E94F7
:103BC0005A1A8091490E882309F11092490E85E511
:103BD00097E00E946B0820E030E0F901EE0FFF1F34
:103BE000EE5AFF4E80819181F901EE0FFF1FE65BD7
:103BF000F14F918380832F5F3F4F2830310569F764
:103C00000E9406038FE697E00E946B088091930E56
:103C10008823C1F01092930E8DE797E00E946B0805
:103C2000F092840E1092890EE0928A0E10928F0EFE
:103C3000D0937D0EC0937C0E0E9406038FE697E022
:103C40000E946B088091920E882389F01092920E48
:103C50000E9406038FE697E00E946B0808C00E944E
:103C6000C71505C00E94201702C00E94CB161E99DE
:103C7000B8CE8AEA97E00E946B080E94AA00B1CEF3
:103C8000EF92FF920F931F937B018C0120E030E0B5
:103C900040E05FE40E94102188238CF0C801B70146
:103CA00020E030E040E05FE40E94B81F0E94402125
:103CB0009B01AC01205030404040504806C0C80134
:103CC000B7010E9440219B01AC01B901CA011F91BB
:103CD0000F91FF90EF900895A0E0B0E0E2E7FEE1E1
:103CE0000C94BD23DC012B01FA019C91923008F465
:103CF00039C1EB018881823008F433C1943069F412
:103D0000843009F02FC111969C91119789819817E1
:103D100009F428C1A5E1BDE025C1843009F421C121
:103D20008230A9F4923009F01DC19A01AD0188E0FA
:103D3000EA010990AE01E90109929E018150C1F7A3
:103D4000E201898111969C918923818308C1923077
:103D500009F407C112962D903C901397EB018A81CC
:103D60009B811496AD90BD90CD90DC901797EC8020
:103D7000FD800E811F819101281B390BB90137FF8E
:103D800004C066277727621B730B603271050CF045
:103D900061C0121613066CF537014801062E04C0E7
:103DA00096948794779467940A94D2F721E030E050
:103DB00040E050E004C0220F331F441F551F6A9596
:103DC000D2F721503040404050402E213F21402327
:103DD0005123211531054105510521F021E030E045
:103DE00040E050E079018A01E628F72808291929DE
:103DF0003CC0232BD1F1260E371E35014601062E7D
:103E000004C096948794779467940A94D2F721E03B
:103E100030E040E050E004C0220F331F441F551F24
:103E20006A95D2F721503040404050402A213B2132
:103E30004C215D21211531054105510521F021E07D
:103E400030E040E050E059016A01A628B728C828B0
:103E5000D9280BC0821593052CF01C01AA24BB2481
:103E6000650103C0EE24FF24870111969C91D201C5
:103E700011968C91981709F445C0992339F0A8013F
:103E800097012A193B094C095D0906C0A601950155
:103E90002E193F09400B510B57FD08C01182338288
:103EA000228224833583468357831DC081E081832A
:103EB0003382228288279927DC01821B930BA40B73
:103EC000B50B84839583A683B7830DC0220F331F60
:103ED000441F551F248335834683578382819381F2
:103EE0000197938382832481358146815781DA014A
:103EF000C9010197A109B1098F5F9F4FAF4FBF4320
:103F000028F30BC0918333822282EA0CFB1C0C1D28
:103F10001D1DE482F5820683178383E0808324815C
:103F200035814681578157FF1AC0C901AA2797FDDD
:103F3000A095BA2F81709070A070B070569547957B
:103F400037952795822B932BA42BB52B84839583B0
:103F5000A683B78382819381019693838283DF0155
:103F600001C0D201CD01CDB7DEB7E2E10C94D92377
:103F7000A0E2B0E0EEEBFFE10C94C92369837A8301
:103F80008B839C832D833E834F835887E9E0EE2EFD
:103F9000F12CEC0EFD1ECE010196B7010E946922A4
:103FA0008E010F5E1F4FCE010596B8010E94692257
:103FB0008A8991E089278A8BC701B801AE01475EE3
:103FC0005F4F0E946C1E0E949421A096E6E00C9424
:103FD000E523A0E2B0E0EFEEFFE10C94C923698392
:103FE0007A838B839C832D833E834F835887F9E0AC
:103FF000EF2EF12CEC0EFD1ECE010196B7010E94B2
:1040000069228E010F5E1F4FCE010596B8010E94F6
:104010006922C701B801AE01475E5F4F0E946C1E66
:104020000E949421A096E6E00C94E523A0E2B0E083
:10403000ECE1F0E20C94BD2369837A838B839C834B
:104040002D833E834F835887CE010196BE01675F63
:104050007F4F0E946922CE010596BE016F5E7F4FA1
:104060000E9469229985923088F089898230C8F04F
:10407000943019F4823051F404C0843029F4923021
:1040800081F485E19DE0C6C0923049F420E09A8534
:104090008A89981321E02A87CE010996BBC0823015
:1040A00049F420E09A858A89981321E02A8BCE0171
:1040B0004196B0C02D843E844F8458886D887E8898
:1040C0008F88988CEE24FF248701AA24BB246501E5
:1040D00040E050E060E070E0E0E0F0E0C1018170BD
:1040E0009070892BE9F0E60CF71C081D191D9A0148
:1040F000AB012A0D3B1D4C1D5D1D80E090E0A0E052
:10410000B0E0E614F7040805190520F481E090E01A
:10411000A0E0B0E0BA01A901480F591F6A1F7B1F38
:10412000AA0CBB1CCC1CDD1C97FE08C081E090E0F3
:10413000A0E0B0E0A82AB92ACA2ADB2A3196E032E8
:10414000F10549F0660C771C881C991C569447941D
:1041500037942794C3CFFA85EA892B893C898B85CC
:104160009C85280F391F2E5F3F4F17C0CA018170F1
:104170009070892B61F016950795F794E79480E08D
:1041800090E0A0E0B0E8E82AF92A0A2B1B2B7695EC
:104190006795579547952F5F3F4F77FDE7CF0CC049
:1041A000440F551F661F771F17FD4160EE0CFF1C63
:1041B000001F111F21503040403090E0590790E01F
:1041C000690790E4790760F32B8F3C8FDB01CA010C
:1041D0008F779070A070B07080349105A105B10503
:1041E00061F447FD0AC0E114F1040105110529F04D
:1041F000405C5F4F6F4F7F4F40781A8EFE1711F073
:1042000081E08A8F4D8F5E8F6F8F78A383E0898FD7
:10421000CE0149960E949421A096E2E10C94D92304
:10422000A8E1B0E0E6E1F1E20C94C92369837A8366
:104230008B839C832D833E834F83588789E0E82EB0
:10424000F12CEC0EFD1ECE010196B7010E946922F1
:104250008E010F5E1F4FCE010596B8010E946922A4
:104260008985823040F08989823028F0C701B80101
:104270000E94E12201C08FEF6896E6E00C94E523EE
:10428000ACE0B0E0E6E4F1E20C94CD2369837A83FC
:104290008B839C83CE010196BE016B5F7F4F0E9492
:1042A00069228D81823061F1823050F1843021F4B5
:1042B0008E81882351F12EC02F81388537FD20C093
:1042C0006E812F3131051CF06623F9F023C08EE199
:1042D00090E0821B930B29853A854B855C8504C051
:1042E00056954795379527958A95D2F76623B1F06D
:1042F00050954095309521953F4F4F4F5F4F0EC0E1
:1043000020E030E040E050E009C02FEF3FEF4FEFFA
:104310005FE704C020E030E040E050E8B901CA01A6
:104320002C96E2E00C94E923DF92EF92FF920F9338
:104330001F93FC01E480F58006811781D180808184
:10434000823048F480E090E0A0E1B0E0E82AF92A69
:104350000A2B1B2BA5C0843009F49FC0823021F4A6
:10436000EE24FF24870105C0E114F10401051105C5
:1043700019F4E0E0F0E096C0628173819FEF62384B
:1043800079070CF05BC022E83FEF261B370B2A3180
:1043900031052CF020E030E040E050E02AC0B801C8
:1043A000A701022E04C076956795579547950A9404
:1043B000D2F781E090E0A0E0B0E004C0880F991F40
:1043C000AA1FBB1F2A95D2F70197A109B1098E2117
:1043D0009F21A023B1230097A105B10521F081E021
:1043E00090E0A0E0B0E09A01AB01282B392B4A2BDA
:1043F0005B2BDA01C9018F779070A070B0708034A8
:104400009105A105B10539F427FF09C0205C3F4F94
:104410004F4F5F4F04C0215C3F4F4F4F5F4FE0E075
:10442000F0E02030A0E03A07A0E04A07A0E45A07F5
:1044300010F0E1E0F0E079018A0127C060387105F1
:1044400064F5FB01E158FF4FD801C7018F779070E9
:10445000A070B07080349105A105B10539F4E7FE74
:104460000DC080E490E0A0E0B0E004C08FE390E0F5
:10447000A0E0B0E0E80EF91E0A1F1B1F17FF05C0E1
:1044800016950795F794E794319687E0169507956A
:10449000F794E7948A95D1F705C0EE24FF248701AD
:1044A000EFEFF0E06E2F679566276795902F9F7767
:1044B000D794DD24D7948E2F8695492F462B582FDD
:1044C0005D29B701CA011F910F91FF90EF90DF9016
:1044D0000895FC01DB01408151812281622F6F77B9
:1044E00070E0221F2227221F9381892F880F822BA1
:1044F000282F30E0991F9927991F11969C931197A7
:1045000021153105A9F5411551056105710511F414
:1045100082E037C082E89FEF13969C938E931297A8
:104520009A01AB0167E0220F331F441F551F6A95A4
:10453000D1F783E08C930DC0220F331F441F551F0A
:1045400012968D919C911397019713969C938E933D
:104550001297203080E0380780E0480780E4580751
:1045600058F314962D933D934D935C9317970895AC
:104570002F3F310579F4411551056105710519F495
:1045800084E08C93089564FF03C081E08C9312C093
:104590001C9210C02F57304013963C932E931297C5
:1045A00083E08C9387E0440F551F661F771F8A9521
:1045B000D1F7706414964D935D936D937C93179728
:1045C00008951F93DC01FB019C91923008F447C0D1
:1045D0008081823008F443C0943051F411961C91CC
:1045E000843099F58181682F70E0611B71093FC0AB
:1045F000843021F0923031F48230B9F18181882306
:1046000089F12DC011961C9111978230F1F08181B2
:104610001817D9F412962D913C91139782819381AA
:104620008217930794F028173907BCF014968D91E0
:104630009D910D90BC91A02D24813581468157819B
:10464000281739074A075B0718F4112341F00AC0FD
:1046500082179307A407B50740F4112319F061E00E
:1046600070E005C06FEF7FEF02C060E070E0CB014B
:104670001F910895629FD001739FF001829FE00D0A
:10468000F11D649FE00DF11D929FF00D839FF00DD1
:10469000749FF00D659FF00D9927729FB00DE11D7D
:1046A000F91F639FB00DE11DF91FBD01CF0111245A
:1046B0000895AA1BBB1B51E107C0AA1FBB1FA61769
:1046C000B70710F0A61BB70B881F991F5A95A9F7BB
:1046D00080959095BC01CD01089597FB092E072682
:1046E0000AD077FD04D0E5DF06D000201AF47095DB
:1046F00061957F4F0895F6F7909581959F4F0895A6
:10470000A1E21A2EAA1BBB1BFD010DC0AA1FBB1FD5
:10471000EE1FFF1FA217B307E407F50720F0A21B47
:10472000B30BE40BF50B661F771F881F991F1A94B4
:1047300069F760957095809590959B01AC01BD01DE
:10474000CF01089597FB092E05260ED057FD04D002
:10475000D7DF0AD0001C38F450954095309521954C
:104760003F4F4F4F5F4F0895F6F7909580957095A6
:1047700061957F4F8F4F9F4F08952F923F924F9299
:104780005F926F927F928F929F92AF92BF92CF92E1
:10479000DF92EF92FF920F931F93CF93DF93CDB7EA
:1047A000DEB7CA1BDB0B0FB6F894DEBF0FBECDBF62
:1047B00009942A88398848885F846E847D848C8433
:1047C0009B84AA84B984C884DF80EE80FD800C813C
:1047D0001B81AA81B981CE0FD11D0FB6F894DEBF1F
:1047E0000FBECDBFED010895662777270C9458249E
:1047F000FC0188279927E89421912032E9F3293098
:1048000010F02E30C8F32B3241F02D3239F4689479
:1048100004C00E942824820F911D219120532A3028
:10482000C0F31EF4909581959F4F0895FB01DC0124
:104830000D900020E9F7119701900D920020E1F70B
:104840000895FB01DC0101900D920020E1F708952D
:104850007AE0979F902D879F802D910D11240895C8
:10486000DC01CB01FC01F999FECF06C0F2BDE1BD30
:10487000F89A319600B40D9241505040B8F708951F
:10488000DC01CB0103C02D910E944B2441505040CC
:10489000D0F70895262FF999FECF1FBA92BD81BD9A
:1048A00020BD0FB6F894FA9AF99A0FBE01960895B2
:1048B0008F929F92AF92BF92CF92DF92EF92FF9230
:1048C0000F931F93CF93DF93EC015B01611571058B
:1048D00019F0FB0191838083F9908F2D90E00E9465
:1048E000C625892BC9F7FDE2FF1621F4F990EE24C5
:1048F000E39405C02BE2F21609F4F990EE248E0140
:1049000001501040C8016CEC70E043E050E00E94A0
:10491000CE25892B01F58E010E5F1F4FC8016FEC6C
:1049200070E045E050E00E94CE25892B19F48E01FD
:10493000095F1F4FA114B10419F0F5011183008321
:10494000E0FC04C070E090E080E814C070E090E00B
:1049500080E86FEF08C1C80164ED70E043E050E00B
:104960000E94CE25892B69F4A114B10429F470E0CA
:1049700090E080EC6FE7F7C02296F501D183C08309
:10498000F6CF8824992440E050E060E070E0EF2DFD
:10499000E053EA30A0F5F2E0EF2A8E2D90E09C0182
:1049A00028703070E2FE06C0232B79F50894811C34
:1049B000911C2BC0232B19F0089481089108DB016E
:1049C000CA0112E0880F991FAA1FBB1F1A95D1F7C1
:1049D000480F591F6A1F7B1F440F551F661F771F03
:1049E0004E0F511D611D711D483929E9520729E9F2
:1049F000620729E1720748F084E0E82A06C0EE3F2A
:104A000031F4E3FC39C098E0E92AF990C0CFE533EE
:104A100011F0E53189F529912D3219F4E0E1EE2A02
:104A200005C02B3219F081E090E003C0299182E0AB
:104A300090E0E22FE053EA3018F0C81BD90B1CC0FD
:104A400020E030E0FCE020383F075CF4C901880F2B
:104A5000991F880F991F280F391F220F331F2E0F00
:104A6000311DE991E053EA3068F3E4FE03C030956C
:104A700021953F4F820E931ECE2CDD24E1FE07C010
:104A8000A114B10421F02197F501D183C083CB019A
:104A9000BA010E94EA257B018C01F3E0CF22DD24DC
:104AA00023E0C216D10421F417FB109517F91095D5
:104AB00057016801C801B70120E030E040E050E054
:104AC0000E94E625882309F44AC097FE0DC02BEE0C
:104AD000E22E20E0F22E9094819491089394C0E20B
:104AE000D0E000E010E012C093E0E92E91E0F92E52
:104AF000F6CFF7012591359145915491C601B50145
:104B00000E9416205B016C018C1A9D0A8C169D0672
:104B100084F7D595C7950F5F1F4F0630110529F013
:104B20008CEF9FEFE80EF91EF1CFC501D6017C0195
:104B30008D018C2D880F8D2D881F8F3F51F0C60160
:104B4000B50120E030E040E050E00E94E6258823F7
:104B500031F482E290E09093B7108093B6107E2DEE
:104B60009F2D802F612F272F392F482F562FB901C6
:104B7000CA01DF91CF911F910F91FF90EF90DF90CD
:104B8000CF90BF90AF909F908F900895911183C068
:104B9000803219F089508550D0F70895FB01DC016F
:104BA0004150504088F08D9181341CF08B350CF4CD
:104BB000805E659161341CF06B350CF4605E861B81
:104BC000611171F3990B0895881BFCCF40D008F454
:104BD00081E00895E89409C097FB3EF49095809594
:104BE000709561957F4F8F4F9F4F9923A9F0F92FB3
:104BF00096E9BB279395F695879577956795B79531
:104C0000F111F8CFFAF4BB0F11F460FF1BC06F5F16
:104C10007F4F8F4F9F4F16C0882311F096E911C028
:104C2000772321F09EE8872F762F05C0662371F049
:104C300096E8862F70E060E02AF09A95660F771F5D
:104C4000881FDAF7880F9695879597F90895990F39
:104C50000008550FAA0BE0E8FEEF16161706E80746
:104C6000F907C0F012161306E407F50798F0621B67
:104C7000730B840B950B39F40A2661F0232B242B3C
:104C8000252B21F408950A2609F4A140A6958FEF5B
:104C9000811D811D0895992788270895F894FFCFD5
:104CA000526561645F53657475703A20000A0D00A7
:104CB00057726F6E672045454D414749433A200082
:104CC0002F00B40000000000000000000000000001
:104CD00000000000000000000000000000000000D4
:104CE000000000006400640064006400640064006C
:104CF0006400640009120D0810040B0E0214070171
:104D00000F050C0009120D0810040B0E0214070108
:104D10000F050C000A0A0A0A0A0A0A0A0A0A0A0AFB
:104D20000A0A0A0A1414141414141414141414146B
:104D3000141414141E1E1E1E1E1E1E1E1E1E1E1EBB
:104D40001E1E1E1E6464646464646464646464643B
:104D500064646464000102030405060708090A0B81
:104D60000C0D0E0F0E0F14150C100B191A11161234
:104D70000D171318110C1A150F10130B0E180D1612
:104D80001719121414120D0F181316110C1A100BF8
:104D90000E15191716130E140F181510190B0C1ADF
:104DA000120D171115101317120E0C1A0B0F110DEF
:104DB000161814190E0F14150C100B191A111612BF
:104DC0000D17131819110C1A150B140F1810120EB9
:104DD000170D13161613180D170F100B190E1215A9
:104DE00014110C1A0E17120F110C1A1510160B14A1
:104DF00019130D180B0C0D0E0F101112131415169C
:104E00001718191A6009455252310D0A00455252BD
:104E1000320D0A00455252330D0A00455252340DEC
:104E20000A0054454D323A20002E000A0D0050521F
:104E300045323A200043414C493A20003B000305EB
:104E4000080E1A302E382D313331303036303938A3
:104E500034000A0D535953494E464F3A7A696762F6
:104E600069742F72782D70706D2F6D6573686E6523
:104E7000746963732F302E382D3133313030363032
:104E80003938340A0D0053434E003B00200A0D52BE
:104E9000534900200A0D4C514900200A0D4144435A
:104EA00000200A0D43485600200A0D4653560020A4
:104EB0000A0D4554433B00200A0D47505300200A79
:104EC0000D002D2D2D2D2D2D2D2D2D2D2D2D2D2D5F
:104ED0002D2D2D2D2D2D2D2D2D2052434F50454E56
:104EE0003234202D2D2D2D2D2D2D2D2D2D2D2D2DF3
:104EF0002D2D2D2D2D2D2D2D2D2D0A0D00496E66BC
:104F00006F3A2020202020202020205A69676269E3
:104F10007420525820384368616E6E656C2D505075
:104F20004D204F75747075740A0D00537973746554
:104F30006D3A202020202020207A69676269742F32
:104F400072782D70706D2F6D6573686E657469630E
:104F5000732F302E382D31333130303630393834EC
:104F60000A0D004472697665723A202020202020C4
:104F7000200070706D2D6F757420006E61757469FE
:104F80006328004368616E6E656C732D3E536572D5
:104F9000766F2D003B200078007573292000746522
:104FA0006C656D65747269652000202020202020CA
:104FB0002020202020202020200A0D0050726F7415
:104FC0006F636F6C20202020202000647373732097
:104FD000006668737320007468737320006C6973D3
:104FE00074656E2D6265666F72652D74616C6B20E1
:104FF00000525353492864426D293A202020200052
:105000002C002020202020202020202020202020B4
:10501000200A0D4E4F4953452864426D293A2020FD
:1050200020002020202020202020202020202020A0
:10503000200A0D534E2D44696666286442293A20A1
:105040002000202020202020202020202020202080
:10505000200A0D4C51493A202020202020202020D9
:105060002000202020202020202020202020202060
:10507000200A0D4552524F52533A20202020202022
:10508000200028002F00200025292020202020207B
:105090002020202020202020200A0D484F50503A68
:1050A0002020202020202020200020202020202020
:1050B00020202020202020202020200A0D54784964
:1050C000443A2020202020202020200020280029D1
:1050D0002020202020202020202020202020200AE6
:1050E0000D5345513A202020202020202020200050
:1050F0002020202020202020202020200A0D0041D8
:10510000444327733A2020202020202020303D00D7
:1051100020313D0020323D0020333D002020202062
:105120000A0D004F534343414C20202020202020D3
:105130002000202020202020200A0D005461626CD5
:1051400065733A20202020202020002C200056616A
:105150006C7565732020202020202020004C617376
:10516000742D4D756C74694E756D20004D756C74A1
:105170006976616C756573202020002D3E00292022
:1051800000202020202020200A0D4D756C746976A7
:10519000616C756573322020004D543A003A00204E
:1051A000200A0D002D2D2D2D2D2D2D2D2D2D2D2DAC
:1051B0002D2D2D2D2D2D2D2D2D0A0D003E003D00C8
:1051C0004D453A000A0D0072636F70656E32342DE2
:1051D000727820285A6967626974205258203843CF
:1051E00068616E6E656C2D50504D204F75747075F2
:1051F00074290A0D0053657474696E672046616CEA
:1052000065736176652D56616C7565730A0D005383
:10521000657475702D53617665640A0D004D756C6B
:10522000746970726F702D53657474696E67730A58
:105230000D002E2E2E73617665642E2E2E002E2EDE
:105240002E72657365742E2E2E0062696E642E2E8A
:105250002E2E0A0D000103030303000000000000CE
:10526000000003030303030303030404040404040E
:1052700004040404040404040404040404040404EE
:1052800004040202030202030303030203030303F1
:10529000020303030303420E460E470E480E490E57
:1052A0004A0E4C0E4E0E500E520E540E560E580E06
:1052B0005A0E5B0E5C0E5D0E5E0E5F0E600E610E92
:1052C000620E630E640E650E660E670E680E690E42
:1052D0006A0E6B0E6C0E6D0E6E0E6F0E700E710EF2
:1052E000720E730E740E750E760E770E780E790EA2
:1052F0007A0E7C0E7E0E7F0E810E830E840E850E3E
:10530000860E870E890E8A0E8B0E8C0E8D0E8F0EDA
:10531000900E910E920E930E6964007461626C653A
:105320000074696D657461626C65004661696C73D7
:105330006176654D6F6465004661696C7361766581
:10534000536574004661696C7361766556616C756E
:1053500065735F31004661696C7361766556616C97
:105360007565735F32004661696C7361766556617D
:105370006C7565735F33004661696C736176655661
:10538000616C7565735F34004661696C7361766545
:1053900056616C7565735F35004661696C73617643
:1053A0006556616C7565735F36004661696C736143
:1053B000766556616C7565735F37004661696C731D
:1053C00061766556616C7565735F380053657276FA
:1053D0006F4D61705F3100536572766F4D61705F24
:1053E0003200536572766F4D61705F3300536572A2
:1053F000766F4D61705F3400536572766F4D6170EA
:105400005F3500536572766F4D61705F360053658E
:1054100072766F4D61705F3700536572766F4D61C4
:10542000705F3800536572766F4475616C526174B9
:10543000655F3100536572766F4475616C526174BB
:10544000655F3200536572766F4475616C526174AA
:10545000655F3300536572766F4475616C52617499
:10546000655F3400536572766F4475616C52617488
:10547000655F3500536572766F4475616C52617477
:10548000655F3600536572766F4475616C52617466
:10549000655F3700536572766F4475616C52617455
:1054A000655F3800536572766F41747655705F3171
:1054B00000536572766F41747655705F32005365A4
:1054C00072766F41747655705F3300536572766FF4
:1054D00041747655705F3400536572766F4174760F
:1054E00055705F3500536572766F41747655705F05
:1054F0003600536572766F41747655705F3700538E
:105500006572766F41747655705F380053657276B8
:105510006F417476446F776E5F3100536572766FBA
:10552000417476446F776E5F3200536572766F41D7
:105530007476446F776E5F3300536572766F417493
:1055400076446F776E5F3400536572766F41747680
:10555000446F776E5F3500536572766F41747644A1
:105560006F776E5F3600536572766F417476446F65
:10557000776E5F3700536572766F417476446F774C
:105580006E5F380050574D526174655F310050575F
:105590004D526174655F320050504D4368616E6ECC
:1055A000656C730050504D53796E630050504D53ED
:1055B000686966740050504D496E76657274006D6E
:1055C000756C74695F6368616E6E656C006D756C97
:1055D00074695F6368616E6E656C73006D756C7481
:1055E000695F6D73796E635F6E756D006D756C7458
:1055F000695F6D73796E635F6C656E006D756C7459
:10560000695F6368616E6E656C6D6170006D756C6D
:105610007469325F6368616E6E656C006D756C7481
:1056200069325F6368616E6E656C73006D756C7472
:1056300069325F6D73796E635F6E756D006D756C49
:105640007469325F6D73796E635F6C656E006D7542
:105650006C7469325F6368616E6E656C6D61700059
:105660006D656E755F6C656E006373765F6F7574E4
:105670007075740073617665006D756C746973651F
:10568000740078087B0881088B089808A408B5087E
:10569000C608D708E808F9080A091B092C093709C0
:1056A00042094D09580963096E0979098409940969
:1056B000A409B409C409D409E409F409040A110AC3
:1056C0001E0A2B0A380A450A520A5F0A6C0A7B0A2C
:1056D0008A0A990AA80AB70AC60AD50AE40AEE0A8B
:1056E000F80A040B0C0B150B1F0B2D0B3C0B4C0B72
:1056F0005C0B6D0B7C0B8C0B9D0BAE0BC00BC90BAD
:10570000D40BD90B476C6F62616C004661696C7396
:1057100061766500536572766F2D4D61700044753A
:10572000616C72617465004174762D55700041742E
:10573000762D446F776E0050574D2D4F75747075F0
:10574000740050504D2D4F7574707574004D756C0C
:10575000746970726F70004D756C746970726F70DF
:1057600032004D656E7500640C6B0C740C7E0C87FA
:105770000C8E0C970CA20CAD0CB70CC20C00030DD8
:10578000151D252D2F33383D030A0808080802048B
:1057900005050401010101010101010101010101EE
:1057A00001010101010101010101010101010101E9
:0E57B000010101FF01000000000000000000E8
:00000001FF
